:020000000528D1
:08000800B428831617308500AF
:10001000003086000230880007308100831285019D
:100020008601081481010614640021300102031CBA
:10003000142881010310860D031C14288515640003
:1000400021300102031C1F28851112308D0081010F
:100050000B11A0308B0008156400881C2C2809089F
:100060008C008810B5300C02031C86288D0B3928B3
:10007000692864008E01B5300C0203180E14BA30E2
:100080000C0203188E140E0886008E01BF300C027D
:1000900003180E15C4300C0203188E150E088600C6
:1000A0008E01C9300C0203180E16CE300C02031854
:1000B0008E160E0886008E01D3300C0203180E1720
:1000C000D8300C0203188E170E088600881C3928B9
:1000D0002F2864008B138B1B69288B1286018316D3
:1000E0000F3081008312630008140000000008151F
:1000F0000819782888100810B5300902031C8128D7
:10010000732883160730810083128B288B138B1B77
:1001100086280030860081010B118D0164000B1DC3
:100120008E280B118D0A06300D02031C8E288515B2
:100130008101640062300102031C9928851181014C
:10014000640062300102031CA0288515810164004F
:1001500062300102031CA728851181016400C330AD
:0E0160000102031CAE2897280B110815090098
:00000001FF
